:03F0000002F00813
:03F0610002F003B7
:05F0030012F08B80FEFD
:04F06400AA82AB834E
:05F068001ABAFF011BB4
:0EF06D00C3E49A74808BF063F08095F0500F2E
:04F07B007CB07D04E4
:05F07F001CBCFF011D97
:06F08400EC4D70F780DE88
:01F08A002263
:07F08B0090FE00E0FAC2A8AC
:03F0920075E10223
:0EF0950090DF3BE0FBBB0DF87B0090000AC053
:0AF0A30002C00312F064D003D00293
:0EF0AD00C3EB9A500F90DF3AE0FC74806CFBCE
:06F0BB0090FE00F080EC65
:03F0C10075E104F2
:0EF0C40090DF3BE0FBBB01F890DF0074AAF088
:09F0D20090DF0174AAF075E1035E
:0EF0DB0090DF3BE0FBBB13F890000AC002126E
:08F0E900F064D002A502F092D0
:06F03700E478FFF6D8FDAD
:08F015007900E94400601B7A58
:05F01D000090F0F57801
:03F02200007593E3
:0AF0250000E493F2A308B80002050E
:08F02F0093D9F4DAF27593FFA6
:08F03D007800E84400600A7944
:03F04500007593C0
:06F0480000E4F309D8FC0E
:08F04E007800E84400600C7931
:0BF0560000900000E4F0A3D8FCD9FA01
:03F0080075810708
:0AF00B0012F0F1E582600302F00349
:04F0F1007582002202
:00000001FF
